:020000040000FA
:0600000051EF08F01200B0
:0600080004EF0AF01200F3
:060018000CEF0AF01200DB
:0E00200001003E000000BB00000002000000D6
:02002E0000EEE2
:0C00300000F00F0EEE6AEA62FDD712002D
:02003C001200B0
:02003E000100BF
:040044001200120094
:080048003F0E93160001636BEB
:10005000676968696969666B010E6A6F1200D9CFBA
:10006000E6FFE1CFD9FFE652000163511FE1040131
:1000700008BF1BD0400EE66E700EE66E030EE66EF5
:100080008AEC06F0E552E552E5520001010E636F7D
:10009000DF6A400EDF5C09E2DF50EA6AB00FE96E0A
:1000A000030EEA22EF6ADF2AF4D797D103017051D9
:1000B000080A01E181D11F0A01E124D1110A01E1FD
:1000C00019D1030A01E1B5D0010A6AE0070A5DE02F
:1000D000010A01E082D10301020EB06F03013A0E62
:1000E000B16F0301020EB26F0301010EB36F030182
:1000F000B46B140EB56FB66BB76B0301B86B6C0EB7
:10010000B96FBA6BBB6B0301030EBC6F0301BD6B10
:10011000BE6B300EBF6FC06B03010E0EC16FC26BA2
:10012000C36BC46B0301010EC56F0301C66BC76BC4
:10013000200EC86FC96B0301080ECA6FCB6BCC6B66
:10014000CD6B0301CE690301020ECE6F0301CF6BAD
:10015000D06BF00ED16FD26B0301D36B010ED46F55
:10016000D56BD66B0301D76904010CBF0DD0400ECF
:10017000E66EB00EE66E030EE66E50EC06F0E5524B
:10018000E552E5520001636B28D10001010E6A6F50
:100190000301715102E100016A6B0001636B1DD123
:1001A000500E0001646F656B0001000E645D020E6D
:1001B00065591FE2040064C000F065C001F0026AE6
:1001C000060E1F0B00C0F6FF01C0F7FF02C0F8FFCC
:1001D00006E0D890F636F736F836E806FAE1940EDF
:1001E000A66E9ED9DEEC06F00001642B000E65239E
:1001F000DBD7DF6A0400DF50A96EA868040EA66E84
:10020000DEEC06F08DD9DF50DF2A006E016A026A4B
:10021000FF0E005C000E0158000E0258EBE3F66A78
:10022000F76A200EF86E940EA66E7AD90001636B01
:10023000D4D0300E0301735D07E100016A5101E182
:1002400032D90001636BC9D0F00E0301735D04E184
:100250004DD90001636BC1D0E8680001671905E161
:10026000E868681902E1E868691906E171C367F096
:1002700072C368F073C369F0670EE96E000EEA6E30
:10028000EE500301711908E1EE500301721904E107
:10029000EE500301731900E12AE1DF6A0301755191
:1002A000DF5C25E23A0E0301D8807555DF24EA6A47
:1002B000760FE96E030EEA22EF50E66E00016651FA
:1002C000EA6A6B0FE96E000EEA22E552E750EF6E24
:1002D0000001662B0001672B000E6823000E6923C6
:1002E000200E0001665D01E17DD8DF2AD7D700012D
:1002F000636B73D077D80001676968696969000129
:10030000636B6BD00301170EB06F71C3B1F372C38F
:10031000B2F373C3B3F374C3B4F375C3B5F371C36A
:10032000F6FF72C3F7FF73C3F8FFDF6A030175516D
:10033000DF5C31E2F00E0301735D13E1DF50030176
:100340007125A96EA66AA6803A0E0301D88075555C
:10035000DF24EA6AB60FE96E030EEA22A8CFEFFFA8
:1003600018D00900300EF85C08E1050EF65C01E1DA
:10037000F568080EF65C01E1F5683A0E0301D880D5
:100380007555DF24EA6AB60FE96E030EEA22F5CF4F
:10039000EFFFDF2ACBD704010CBF0DD0400EE66E75
:1003A000B00EE66E030EE66E50EC06F0E552E55236
:1003B000E5520001636B11D06D926D6ADF6AFF0E2A
:1003C000DF5C09E2E868E85004E0E80600D000D00D
:1003D000FAD7DF2AF4D7FF0000D0E552E552E7CF85
:1003E000D9FF12000301F16B66C000F0016A026AD6
:1003F00000500001675DF66E015000016859F76E0C
:10040000025000016959F86E1F0EF6140301F26FD5
:10041000E00EF6160301F06B200E0301F05D1FE203
:100420000301F25115E1000166510FE00301F151A2
:10043000EA6A6B0FE96E000EEA22EF50F56E0D00CE
:100440000301F12B0001660702D0F5680D0004D00E
:10045000F5680D000301F2070301F02BDDD70A0058
:10046000A40EA66E5DD80301F06B00016651030176
:10047000F05D18E20301F1510301F025EA6A6B0F08
:10048000E96E000EEA22EF50E66E0301F051EA6ACF
:100490006B0FE96E000EEA22E552E750EF6E0301A2
:1004A000F02BE3D7120071C3F6FF72C3F7FF73C3DB
:1004B000F8FF0301F36B030175510301F35D15E2CE
:1004C0003A0E0301D88075550301F325EA6A760FC9
:1004D000E96E030EEA22EF50F56E0C00C40EA66E14
:1004E0001FD809000301F32BE6D712000301F46BB8
:1004F0007551F45D14E27151F425A96E3A0ED8805D
:100500007555F425EA6A760FE96E030EEA22EF507C
:10051000A86E040EA66E04D80301F42BE9D71200CE
:10052000F29E550EA76EAA0EA76EA682A6B2FED7A1
:04053000A69412007B
:0C053400D9CFE6FFE1CFD9FFE6526C50B2
:1005400032E16896040100513C0BE842E8420D0894
:1005500028E1180E021923E1040E031920E1100E00
:10056000026F040E036FDF6ADF50006E016A080E2F
:10057000005C000E015813E2DF50EA6A180FE96EC2
:10058000040EEA22EF50E66EDF50EA6A100FE96EC1
:10059000040EEA22E552E750EF6EDF2AE5D711D8C4
:1005A0000AD048D808D0040E6C5C03E168965FD886
:1005B00002D0000E01D0010EE552E552E7CFD9FF7F
:1005C0001200D9CFE6FFE1CFD9FFE652040104BF04
:1005D000046B0001B36BAB6BAC6BB16BB26B55ECE6
:1005E00004F0DF6ADF50006E016A010E005C000E4D
:1005F00001581AE20001AC5117E1F76ADF34FE0B33
:10060000F736F66E8A0EF6260F0EF7220900F5CFA2
:1006100000F00800F5CF01F004D001C0FAFF00504F
:10062000F96EFBDFDF2ADED7F6D8E552E552E7CFD9
:10063000D9FF1200020E0001AB5D0EE1AFD804013C
:10064000180E026F040E036F080E016F00BD02D07A
:10065000C80E0BD0880E09D023D90401080E016FF3
:10066000100E026F040E036F8C0E006F1200040E4A
:100670000001B45D09E112C46EFF6E50000802E291
:10068000050E01D0030EB46F0001AB0510E111D8C7
:10069000020E0001B35D03E10401840E06D00401E3
:1006A00004BD02D0C80E01D0880E046F120050EFB6
:1006B00004F0D9CFE6FFE1CFD9FF020EE126000119
:1006C000080EB15D000EB2590DE2B1C0DEFFB2C03E
:1006D000DDFFB35102E1010E03D0B30506E1020EC6
:1006E000B36F03D0080EDE6EDD6A0401049304913B
:1006F000010EDB500413DFCF05F4000EDB500001C8
:10070000B15F010EDB50B25B180EAF6F040EB06F1D
:100710000001B5A31DD0D9CFE9FFDACFEAFFEE5033
:10072000ED1032E0ADC0F6FFAEC0F7FF0800F550A7
:10073000AFC0E9FFB0C0EAFFEF6E0001AF2B000EC3
:10074000B023AD2BAE23DF06010EE5E2DB06E3D7D7
:10075000D9CFE9FFDACFEAFFEE50ED1015E0ADC0DA
:10076000E9FFAEC0EAFFEF50AFC0E9FFB0C0EAFF5B
:10077000EF6E0001AF2B000EB023AD2BAE23DF06D2
:10078000010EE6E2DB06E4D7020EE15C02E2E16A7A
:10079000E552E16EE552E7CFD9FF1200D9CFE6FF6F
:1007A000E1CFD9FF020EE126030E04010015E76E2A
:1007B000010EE7CFDBFF01C4DFFFDE500001B127F0
:1007C000DD50B223180EAD6F040EAE6FD9CFE9FF26
:1007D000DACFEAFFEE50ED1014E0ADC0E9FFAEC095
:1007E000EAFFEF50AFC0E9FFB0C0EAFFEF6EAF2BFA
:1007F000000EB023AD2BAE23DF06010EE7E2DB06D1
:10080000E5D7020EE15C02E2E16AE552E16EE552F3
:10081000E7CFD9FF12006D980001AC510BE1040144
:10082000080E016F100E026F040E036F840E006F2E
:10083000040123D0040110AF22D00001B151040102
:10084000165D0001B2510401175904E216C4B1F05B
:1008500017C4B2F02EDF0001010EAB6F0401080EC9
:10086000016F100E026F040E036F800E006F040103
:10087000180E066F040E076FC80E046F12000001F9
:10088000020EAB6F0401056BC80E046F0401080E65
:10089000016F180E026F040E036FC80E006F120076
:0A08A0000001AB6B0401046B1200B1
:0608AA0004011051600B77
:1008B000E842E842E842E842E842000901E012006A
:1008C0001151070A4CE00B0A4AE0070A3BE0010A13
:1008D00027E00B0A23E0020A21E0030A1DE0080AD0
:1008E00012E0010A0EE00F0A0AE0030A01E012001A
:1008F0000001010EAC6F0001040EB46F1200B0EFE6
:1009000004F007EF05F00001010EAC6F0001B60E18
:10091000AD6F000EAE6F10D02EEF05F079EF05F041
:100920000001010EAC6F040114510001AD6FAE6BFC
:10093000B70EAD27000EAE230001B5930001010EE6
:10094000B16F12000001010EAC6F04011451EA6A8C
:10095000B70FE96E000EEA2212C4EFFF1200120078
:10096000800E0401105D52E11351030A30E0010AC8
:100970000CE0030A49E10001010EAC6F0001CA0E50
:10098000AD6F0E0EAE6F120E3CD00001010EAC6FBB
:1009900004011251F66EF76AD890F636F736800EDB
:1009A000F6260F0EF7220900F5CFADF00A00F5CFBD
:1009B000AEF0020E0001F76AAD25F66EAE51F722D9
:1009C0000900F5CFB1F00A00F5CFB2F01DD000015B
:1009D000010EAC6F04011251F66EF76AD890F6362C
:1009E000F736840EF6260F0EF7220900F5CFADF08C
:1009F0000A00F5CFAEF0ADC0F6FFAEC0F7FF0800BD
:100A0000F5500001B16FB26B0001B5831200000117
:100A1000010EAC6F0F0EE66E710EE66E0F0EE66EF7
:100A200050EC07F0E552E552E552010EE66EB70EC6
:100A3000E66E000EE66E50EC07F0E552E552E55228
:100A400012C4B6F00401125104E10001050EB46FA6
:100A500012000001060EB46F3BEF06F00401186BA4
:100A6000196B040110511F0B020A13E0030A0DE079
:100A7000010A31E10001010EAC6F0401188100018F
:100A8000B5A129D00401188326D00001010EAC6F56
:100A900022D00001010EAC6F040114510F0B080DA0
:100AA000F350016A000F006E040E01221451800BF6
:100AB00001E0010E040DF35000010024AF6F000EA1
:100AC0000120B06FAFC0E9FFEA6EEF50040B03E006
:100AD0000401010E186F0001AC050AE10001180EB7
:100AE000AD6F040EAE6F0001B5930001020EB16F41
:100AF00012000401120510E110511F0B00090CE156
:100B00000001010EAC6F030E0401115D03E1000151
:100B1000B58102D00001B5910401125136E11051A6
:100B20001F0B020832E114510F0B00092EE00001E7
:100B3000010EAC6F040114510F0B080DF350016A44
:100B4000000F006E040E01221451800B01E0010E13
:100B5000040DF35000010024AF6F000E0120B06FB0
:100B6000030E0401115D02E1840E03D014AF07D01F
:100B7000400EAFC0E9FFB0C0EAFFEF6E1200880E72
:0C0B8000AFC0E9FFB0C0EAFFEF6E12004A
:040B8C0004011051FF
:100B90001F0B010801E01200145101E01200060EC3
:100BA000115D28E11351230A23E0010A0FE0030A33
:100BB0001FE10001020EAC6F0001B60505E1000166
:100BC000EE0EAD6F0E0EAE6F090E0FD00001020ECD
:100BD000AC6F0001B60505E10001630EAD6F0F0EAD
:100BE000AE6F0001B60504E11D0E0001B16FB26BDE
:100BF0000001B58304011051600BE842E842E8426D
:100C0000E842E842010801E0120011510B0A2BE012
:100C1000080A1BE0090A13E0080A09E00B0A05E0CC
:100C2000080A01E0120039EF06F03AEF06F0000181
:100C3000020EAC6F0001B80EAD6F000E0DD00001BA
:100C4000020EAC6F13C4B8F012000001020EAC6FBC
:100C50000001B90EAD6F000EAE6F0001B59300013B
:100C6000010EB16F12000001020EAC6F12C4B9F098
:100C70001200120012000001BA6B1E0E716E040108
:100C8000400E096F200E0A6F040E0B6F880E086F5E
:100C90000401600E0E6F040E0F6F400E0C6F1200F9
:100CA000D9CFE6FFE1CFD9FFE652FC0EDB5040087A
:100CB00005E2400EF36EFC0EF3CFDBFFDF6AFC0EA5
:100CC000DB50DF5C19E2DF50E76EFD0EDBCFE9FFA2
:100CD000FE0EDBCFEAFFE750E926000EEA22EF50D6
:100CE000E66EDF50EA6A600FE96E040EEA22E55212
:100CF000E750EF6EDF2AE3D7FC0EDBCF0DF4400E9A
:100D000004010C170C7D880E0C13E552E552E7CF59
:100D1000D9FF1200D9CFE6FFE1CFD9FF0001BA6BAE
:100D2000040108BF30D0FC0EDBCF00F00951D880A1
:100D3000005403E2FC0E09C4DBFF0001BA6BFC0E99
:100D4000DB50BA5D19E2BA51EA6A200FE96E040E6F
:100D5000EA22EF50E66EBA51E76EFD0EDBCFE9FFF7
:100D6000FE0EDBCFEAFFE750E926000EEA22E5524D
:100D7000E750EF6EBA2BE3D70401400E096F081756
:100D8000087D880E08130001BA51E552E7CFD9FF5C
:020D900012004F
:0E0D92006DA60CD80001B40508E16DBA06D0BC
:100DA000686A696A69806988020EB46F12006D6AA8
:100DB000696A6D860001010EB46F12000001B45122
:100DC00001E1120068B425D86DB2120068B038D8BD
:100DD00068B817D868BA24D8030E0001B45D01E2E0
:100DE00012000301FF6B040EFF5D0AE268A608D043
:100DF0009AEC02F0000901E168960301FF2BF3D79A
:100E00001200698468986D82A19AA08A0300A09A52
:100E100012006D92699468A402D06894FCD7120005
:100E200070A00CD0800E0401005D07E1840E040167
:100E3000045D03E104018C0E006F7090689A12004B
:100E40006A6A686A9F0E6B6E7B0E696E6E6A0F0E21
:100E5000E66E710EE66E0F0EE66E22D8E552E55292
:100E6000E552160E706E68A605D0689600D000D0C8
:100E70000000F9D76D9850EC04F00401080E016FE2
:100E80000401100E026F040E036F04018C0E006F3C
:100E90000001B5910001B66B0001030EB46F1200A2
:100EA000D9CFE6FFE1CFD9FFFD0EDBCFE9FFFE0E84
:100EB000DBCFEAFFFC0EDB5004E0EE6AFC0EDB0643
:0A0EC000F9D7E552E7CFD9FF120081
:060ECA001201000200000D
:100ED0000008D8043C0002000102000109022900B8
:100EE000010100C0320904000002030000000921D2
:100EF00011010001221D00070581034000010705C3
:100F000001034000010403090434034D0069006338
:100F10000072006F006300680069007000200054D8
:100F2000006500630068006E006F006C006F006772
:100F3000007900200049006E0063002E002603485F
:100F400000490044002000550053004200200042A8
:100F5000006F006F0074006C006F0061006400653A
:100F60000072000600FF0901A101190129401500C6
:100F700026FF00750895408100190129409100C0A5
:0C0F8000DC0EDC0E050F090F3D0F8C0B82
:040F8C00200EF66ECF
:100F9000000EF76E000EF86E03010900F550FA6FAF
:100FA0000900F550FB6F03E1FA6701D03DD009005D
:100FB000F550F56F0900F550F66F0900F550F76F21
:100FC00009000900F550E96E0900F550EA6E0900C4
:100FD00009000900F550F86F0900F550F96F090094
:100FE0000900F6CFFCF3F7CFFDF3F8CFFEF3F5C31E
:100FF000F6FFF6C3F7FFF7C3F8FF0301F85302E16A
:10100000F95307E00900F550EE6EF807F8E2F9072A
:10101000F9D7FCC3F6FFFDC3F7FFFEC3F8FF0301DA
:0A102000FA07000EFB5BBFD71200B9
:06102A000F0EC16E81B83B
:1010300004D0070EC16E00EF0AF01DD80ED80400D0
:1010400016D819D8060E0001B45D05E16D50020BEB
:1010500002E12FEC00F0F3D71200140E6F6E0001C6
:10106000B46B0001B56B0001B66B24EF00F0C9EC66
:1010700006F0DEEF06F00001BB51BC1104E1100EDA
:10108000BB6F270EBC6FBB07000EBC5BBB51BC1116
:1010900007E18A7E8A50800B02E08A9C12008A8CCB
:0210A00012003C
:0E10A20013EE00F023EE00F0F86A049CC6EC9A
:0E10B00007F01EEC00F015EC08F0FBD7120064
:1013000013EE00F0000023EE00F00000F86A049CE9
:101310003BEC08F02DEC08F0040037EC08F03BEC57
:1013200008F0060E0001B45D05E16D50020B02E10C
:081330002FEC00F0F1D71200D0
:020000040030CA
:0100000021DE
:010001000EF0
:010002002ECF
:0100030013E9
:01000500807A
:010006008178
:010008000FE8
:01000900C036
:01000A000FE6
:01000B00E014
:01000C000FE4
:01000D0040B2
:00000001FF
